:100000008A110A120528000009000730990083169A
:10001000051085100511051285158312AE01051016
:1000200085100511051285126430A000A10114226B
:1000300005150130AC002C080A3C031C2828E830C8
:10004000A0000330A10014220130AC07031C1B28C0
:100050001F30830505112C30A0000130A1001422AF
:10006000C120AC012C080A3C031C4B280130AD0018
:100070002D083C3C031C4528E830A0000330A100BB
:1000800014220130AD07031C38281F3083050130CE
:10009000AC07031C32281F3083050130AE002E0848
:1000A000013C031D6C28AE010130AC002C08033C60
:1000B000031C692885195E280130AE001F308305B6
:1000C000E830A0000330A10014220130AC07031C6B
:1000D00056281F3083054F281F3083050515013032
:1000E000AC002C080A3C031C7E28E830A00003303A
:1000F000A10014220130AC07031C71281F308305B6
:100100000511AC012C080A3C031C9B280130AD00F2
:100110002D083C3C031C9528E830A0000330A100CA
:1001200014220130AD07031C88281F3083050130DD
:10013000AC07031C82281F3083050130AE002E0857
:10014000013C031DBC28AE010130AC002C08053C6D
:10015000031CB9288519AE280130AE001F30830575
:10016000E830A0000330A10014220130AC07031CCA
:10017000A6281F3083059F281F308305C120312802
:10018000C02805149030A0000130A10014221221D3
:10019000BC213521BC217021BC210921BC21ED20CD
:1001A000CA21ED20BC210121BC21E520BC2109216F
:1001B000BC21E520BC212B21BC210621BC21C8305B
:1001C000A000A101142205100800E021F12108007F
:1001D000F121E021E021E0210800F121E021F121DD
:1001E000E0210800F121E021E0210800E0210800E1
:1001F000E021E021F121E0210800F121F121E021BD
:100200000800E021E021E021E0210800E021E021D8
:100210000800E021F121F121F1210800F121E02184
:10022000F1210800E021F121E021E0210800F12185
:10023000F1210800F121E0210800F121F121F12153
:100240000800E021F121F121E0210800F121F12154
:10025000E021F1210800E021F121E0210800E02166
:10026000E021E0210800F1210800E021E021F12156
:100270000800E021E021E021E021F1210800E02157
:10028000F121F1210800F121E021E021F121080014
:10029000F121E021F121F1210800F121F121E021FA
:1002A000E0210800F121F121F121F121F1210800E3
:1002B000E021F121F121F121F1210800E021E021EB
:1002C000F121F121F1210800E021E021E021F121DB
:1002D000F1210800E021E021E021E021F1210800E6
:1002E000E021E021E021E021E0210800F121E021EE
:1002F000E021E021E0210800F121F121E021E021CD
:10030000E0210800F121F121F121E021E0210800A4
:10031000F121F121F121F121E0210800E021F12179
:10032000E021F121E021F1210800F121F121E0217A
:10033000E021F121F1210800E021E021F121F1216A
:10034000E021E0210800F121E021E021F121E0217C
:100350000800F121E021E021E021F1210800F12154
:10036000E021E021E021E021F121080005125030D8
:10037000A000A1011422080005125030A000A10124
:1003800014225030A000A10114225030A000A1017D
:100390001422080005125030A000A1011422503090
:1003A000A000A10114225030A000A101142250305D
:1003B000A000A10114225030A000A10114220800C5
:1003C0000516053084000230AA009930A0000230E2
:1003D000A1003530A2000030A3004F220512B62143
:1003E00008000516053084000230AA009930A000EC
:1003F0000230A1009E30A2000030A3004F2205125F
:10040000B62108000516053084000230AA00993094
:10041000A0000230A100CB30A2000830A3004F2280
:100420000512B6210800132AA00803191F2A262244
:10043000A00300000000000000000000142AA10832
:10044000031908002622A103A003142A0C30A500DA
:10045000A50B282A000000001230A200A20B352AAA
:100460003722372200000000080037222E2A0D30E4
:10047000A400A40B392A000008001030A8020001D3
:10048000031C013EA902031C0800462A0A30A802E8
:100490000001031C013EA902031C0800462A2A0889
:1004A00080042008A8002108A9003D220130A202F2
:1004B000031CA3032A0980052008A8002108A9001D
:1004C0003D22A208031D4F2AA308031D4F2A08003E
:02400E00C431BB
:00000001FF
